 HlfViewer

 Timestamp is 537255c6 (Tue May 13 21:26:30 2014)

 Preferred load address is 0000000180000000

 Start         Length     Name                   Class
 0001:00000000 00000088H .idata$5                CODE
 0001:00000090 000002d6H .rdata                  CODE
 0001:00000370 00003103H .text                   CODE
 0001:00003478 0000038cH .xdata                  CODE
 0001:00003804 00000028H .idata$2                CODE
 0001:0000382c 00000014H .idata$3                CODE
 0001:00003840 00000088H .idata$4                CODE
 0001:000038c8 00000102H .idata$6                CODE
 0001:000039d0 000000c5H .edata                  CODE
 0002:00000000 0000011cH .data                   DATA
 0002:00000120 00000f70H .bss                    DATA
 0003:00000000 0000033cH .pdata                  DATA
 0004:00000000 00000058H .rsrc$01                DATA
 0004:00000060 00000378H .rsrc$02                DATA

  Address         Publics by Value              Rva+Base               Lib:Object

 0000:00000000       ___safe_se_handler_count   0000000000000000     <absolute>
 0000:00000000       ___safe_se_handler_table   0000000000000000     <absolute>
 0000:00000000       __ImageBase                0000000180000000     <linker-defined>
 0001:00000000       __imp_lstrcpynW            0000000180001000     kernel32:KERNEL32.dll
 0001:00000008       __imp_GetFileAttributesW   0000000180001008     kernel32:KERNEL32.dll
 0001:00000010       __imp_lstrlenW             0000000180001010     kernel32:KERNEL32.dll
 0001:00000018       __imp_lstrcpyW             0000000180001018     kernel32:KERNEL32.dll
 0001:00000020       __imp_DeleteFileW          0000000180001020     kernel32:KERNEL32.dll
 0001:00000028       __imp_CloseHandle          0000000180001028     kernel32:KERNEL32.dll
 0001:00000030       __imp_WriteFile            0000000180001030     kernel32:KERNEL32.dll
 0001:00000038       __imp_CreateFileW          0000000180001038     kernel32:KERNEL32.dll
 0001:00000040       __imp_lstrcatW             0000000180001040     kernel32:KERNEL32.dll
 0001:00000048       __imp_GetFullPathNameW     0000000180001048     kernel32:KERNEL32.dll
 0001:00000050       __imp_ExpandEnvironmentStringsW 0000000180001050     kernel32:KERNEL32.dll
 0001:00000058       __imp_HeapFree             0000000180001058     kernel32:KERNEL32.dll
 0001:00000060       __imp_GetProcessHeap       0000000180001060     kernel32:KERNEL32.dll
 0001:00000068       __imp_HeapAlloc            0000000180001068     kernel32:KERNEL32.dll
 0001:00000070       \177KERNEL32_NULL_THUNK_DATA 0000000180001070     kernel32:KERNEL32.dll
 0001:00000078       __imp_UuidFromStringW      0000000180001078     rpcrt4:RPCRT4.dll
 0001:00000080       \177RPCRT4_NULL_THUNK_DATA 0000000180001080     rpcrt4:RPCRT4.dll
 0001:00000090       MainGuid                   0000000180001090     HlfViewer.obj
 0001:000000a0       MenuGuid                   00000001800010a0     HlfViewer.obj
 0001:000000b0       DialogGuid                 00000001800010b0     HlfViewer.obj
 0001:000000c0       ??_C@_1DE@BGKMIKPD@?$AAE?$AAu?$AAg?$AAe?$AAn?$AAe?$AA?5?$AAR?$AAo?$AAs?$AAh?$AAa?$AAl?$AA?5?$AA?$CG?$AA?5?$AAF?$AAa?$AAr?$AA?5?$AAG?$AAr?$AAo?$AAu?$AAp?$AA?$AA@ 00000001800010c0     HlfViewer.obj
 0001:00000100       ??_C@_1EA@CONHECGE@?$AAH?$AAl?$AAf?$AA?9?$AAf?$AAi?$AAl?$AAe?$AA?5?$AAV?$AAi?$AAe?$AAw?$AAe?$AAr?$AA?5?$AAf?$AAo?$AAr?$AA?5?$AAF?$AAa?$AAr?$AA?5?$AAM?$AAa?$AAn?$AAa?$AAg?$AAe?$AAr?$AA?$AA@ 0000000180001100     HlfViewer.obj
 0001:00000140       ??_C@_1BE@KLINDABO@?$AAH?$AAl?$AAf?$AAV?$AAi?$AAe?$AAw?$AAe?$AAr?$AA?$AA@ 0000000180001140     HlfViewer.obj
 0001:00000158       ??_C@_17KGEADEDI@?$AAH?$AAL?$AAF?$AA?$AA@ 0000000180001158     HlfViewer.obj
 0001:00000160       ??_C@_1M@EFMNOFJK@?$AA?$CK?$AA?4?$AAh?$AAl?$AAf?$AA?$AA@ 0000000180001160     HlfViewer.obj
 0001:00000170       ??_C@_1BC@KGOLMJNA@?$AAM?$AAa?$AAs?$AAk?$AAF?$AAi?$AAl?$AAe?$AA?$AA@ 0000000180001170     HlfViewer.obj
 0001:00000188       ??_C@_1BM@GGPBEDKL@?$AAC?$AAh?$AAe?$AAc?$AAk?$AAM?$AAa?$AAs?$AAk?$AAF?$AAi?$AAl?$AAe?$AA?$AA@ 0000000180001188     HlfViewer.obj
 0001:000001a8       ??_C@_1M@PALMNGCF@?$AAS?$AAt?$AAy?$AAl?$AAe?$AA?$AA@ 00000001800011a8     HlfViewer.obj
 0001:000001b8       ??_C@_1CG@GFFDAIMK@?$AAP?$AAr?$AAo?$AAc?$AAe?$AAs?$AAs?$AAE?$AAd?$AAi?$AAt?$AAo?$AAr?$AAI?$AAn?$AAp?$AAu?$AAt?$AA?$AA@ 00000001800011b8     HlfViewer.obj
 0001:000001e0       ??_C@_15NPKLCIOJ@?$AAF?$AA1?$AA?$AA@ 00000001800011e0     HlfViewer.obj
 0001:000001e8       ??_C@_1BE@IHEBLNLC@?$AAE?$AAd?$AAi?$AAt?$AAo?$AAr?$AAK?$AAe?$AAy?$AA?$AA@ 00000001800011e8     HlfViewer.obj
 0001:00000200       ??_7?$DialogItemBinding@UFarDialogItem@@@@6B@ 0000000180001200     HlfViewer.obj
 0001:00000210       ??_7?$DialogBuilderBase@UFarDialogItem@@@@6B@ 0000000180001210     HlfViewer.obj
 0001:00000258       ??_7PluginEditFieldBinding@@6B@ 0000000180001258     HlfViewer.obj
 0001:00000270       ??_7PluginDialogBuilder@@6B@ 0000000180001270     HlfViewer.obj
 0001:000002b8       ??_7PluginCheckBoxBinding@@6B@ 00000001800012b8     HlfViewer.obj
 0001:000002c8       ??_7PluginRadioButtonBinding@@6B@ 00000001800012c8     HlfViewer.obj
 0001:000002d8       ??_C@_15EFLNJKHH@?$AA?$CF?$AAu?$AA?$AA@ 00000001800012d8     HlfViewer.obj
 0001:000002e0       ??_7PluginIntEditFieldBinding@@6B@ 00000001800012e0     HlfViewer.obj
 0001:000002f0       ??_7PluginUIntEditFieldBinding@@6B@ 00000001800012f0     HlfViewer.obj
 0001:00000300       ??_C@_15JNBOKNOG@?$AA?$AN?$AA?6?$AA?$AA@ 0000000180001300     HlfViewer.obj
 0001:00000308       ??_C@_19CPJEHIBK@?$AA?4?$AAh?$AAl?$AAf?$AA?$AA@ 0000000180001308     HlfViewer.obj
 0001:00000318       ??_C@_1BG@IOFJDEI@?$AA?4?$AAL?$AAa?$AAn?$AAg?$AAu?$AAa?$AAg?$AAe?$AA?$DN?$AA?$AA@ 0000000180001318     HlfViewer.obj
 0001:00000330       ??_C@_11LOCGONAA@?$AA?$AA@ 0000000180001330     HlfViewer.obj
 0001:00000338       ??_C@_17MEJHPLBO@?$AAc?$AAm?$AAd?$AA?$AA@ 0000000180001338     HlfViewer.obj
 0001:00000340       ??_C@_1BE@BAOBMOBE@?$AA?$CF?$AAF?$AAA?$AAR?$AAH?$AAO?$AAM?$AAE?$AA?$CF?$AA?$AA@ 0000000180001340     HlfViewer.obj
 0001:00000354       ??_C@_13FPGAJAPJ@?$AA?2?$AA?$AA@ 0000000180001354     HlfViewer.obj
 0001:00000358       ??_C@_1O@BJPKKLLM@?$AAC?$AAo?$AAn?$AAf?$AAi?$AAg?$AA?$AA@ 0000000180001358     HlfViewer.obj
 0001:00000380       __chkstk                   0000000180001380 f   chkstk.obj
 0001:00000380       _alloca_probe              0000000180001380     chkstk.obj
 0001:000003d0       ?GetLangString@PluginDialogBuilder@@MEAAPEB_WH@Z 00000001800013d0 f i HlfViewer.obj
 0001:000003e0       ?CheckExtension@@YAHPEB_W@Z 00000001800013e0 f   HlfViewer.obj
 0001:00000420       GetGlobalInfoW             0000000180001420 f   HlfViewer.obj
 0001:000004a0       GetPluginInfoW             00000001800014a0 f   HlfViewer.obj
 0001:00000540       ?GetEditorFileName@@YAPEA_WXZ 0000000180001540 f   HlfViewer.obj
 0001:000005c0       ?FindTopic@@YAPEB_W_N0@Z   00000001800015c0 f   HlfViewer.obj
 0001:00000810       ?FindPluginHelp@@YA_NPEB_WPEA_W@Z 0000000180001810 f   HlfViewer.obj
 0001:000009e0       ?GetPluginConfig@@YAXXZ    00000001800019e0 f   HlfViewer.obj
 0001:00000c40       ?InitDialogItem@?$DialogBuilderBase@UFarDialogItem@@@@MEAAXPEAUFarDialogItem@@PEB_W@Z 0000000180001c40 f i HlfViewer.obj
 0001:00000c40       ?SaveValue@?$DialogItemBinding@UFarDialogItem@@@@UEAAXPEAUFarDialogItem@@H@Z 0000000180001c40 f i HlfViewer.obj
 0001:00000c50       ?TextWidth@?$DialogBuilderBase@UFarDialogItem@@@@MEAAHAEBUFarDialogItem@@@Z 0000000180001c50 f i HlfViewer.obj
 0001:00000c60       ?DoShowDialog@?$DialogBuilderBase@UFarDialogItem@@@@MEAA_JXZ 0000000180001c60 f i HlfViewer.obj
 0001:00000c70       ??1?$DialogBuilderBase@UFarDialogItem@@@@MEAA@XZ 0000000180001c70 f i HlfViewer.obj
 0001:00000cf0       ?AddUIntEditField@?$DialogBuilderBase@UFarDialogItem@@@@UEAAPEAUFarDialogItem@@PEAIH@Z 0000000180001cf0 f i HlfViewer.obj
 0001:00000cf0       ?CreateCheckBoxBinding@?$DialogBuilderBase@UFarDialogItem@@@@MEAAPEAU?$DialogItemBinding@UFarDialogItem@@@@PEAHH@Z 0000000180001cf0 f i HlfViewer.obj
 0001:00000cf0       ?CreateRadioButtonBinding@?$DialogBuilderBase@UFarDialogItem@@@@MEAAPEAU?$DialogItemBinding@UFarDialogItem@@@@PEAH@Z 0000000180001cf0 f i HlfViewer.obj
 0001:00000cf0       ?GetLangString@?$DialogBuilderBase@UFarDialogItem@@@@MEAAPEB_WH@Z 0000000180001cf0 f i HlfViewer.obj
 0001:00000cf0       ?AddIntEditField@?$DialogBuilderBase@UFarDialogItem@@@@UEAAPEAUFarDialogItem@@PEAHH@Z 0000000180001cf0 f i HlfViewer.obj
 0001:00000d00       ??_EPluginEditFieldBinding@@UEAAPEAXI@Z 0000000180001d00 f i HlfViewer.obj
 0001:00000d00       ??_EPluginCheckBoxBinding@@UEAAPEAXI@Z 0000000180001d00 f i HlfViewer.obj
 0001:00000d00       ??_GPluginCheckBoxBinding@@UEAAPEAXI@Z 0000000180001d00 f i HlfViewer.obj
 0001:00000d00       ??_EPluginUIntEditFieldBinding@@UEAAPEAXI@Z 0000000180001d00 f i HlfViewer.obj
 0001:00000d00       ??_EPluginRadioButtonBinding@@UEAAPEAXI@Z 0000000180001d00 f i HlfViewer.obj
 0001:00000d00       ??_G?$DialogItemBinding@UFarDialogItem@@@@UEAAPEAXI@Z 0000000180001d00 f i HlfViewer.obj
 0001:00000d00       ??_GPluginIntEditFieldBinding@@UEAAPEAXI@Z 0000000180001d00 f i HlfViewer.obj
 0001:00000d00       ??_GPluginUIntEditFieldBinding@@UEAAPEAXI@Z 0000000180001d00 f i HlfViewer.obj
 0001:00000d00       ??_EPluginIntEditFieldBinding@@UEAAPEAXI@Z 0000000180001d00 f i HlfViewer.obj
 0001:00000d00       ??_E?$DialogItemBinding@UFarDialogItem@@@@UEAAPEAXI@Z 0000000180001d00 f i HlfViewer.obj
 0001:00000d00       ??_GPluginEditFieldBinding@@UEAAPEAXI@Z 0000000180001d00 f i HlfViewer.obj
 0001:00000d00       ??_GPluginRadioButtonBinding@@UEAAPEAXI@Z 0000000180001d00 f i HlfViewer.obj
 0001:00000d30       ??_E?$DialogBuilderBase@UFarDialogItem@@@@MEAAPEAXI@Z 0000000180001d30 f i HlfViewer.obj
 0001:00000d30       ??_G?$DialogBuilderBase@UFarDialogItem@@@@MEAAPEAXI@Z 0000000180001d30 f i HlfViewer.obj
 0001:00000d60       ?ReallocDialogItems@?$DialogBuilderBase@UFarDialogItem@@@@IEAAXXZ 0000000180001d60 f i HlfViewer.obj
 0001:00000e80       ?MaxTextWidth@?$DialogBuilderBase@UFarDialogItem@@@@IEAA_JXZ 0000000180001e80 f i HlfViewer.obj
 0001:00000fa0       ?SaveValue@PluginEditFieldBinding@@UEAAXPEAUFarDialogItem@@H@Z 0000000180001fa0 f i HlfViewer.obj
 0001:00000fe0       ?InitDialogItem@PluginDialogBuilder@@MEAAXPEAUFarDialogItem@@PEB_W@Z 0000000180001fe0 f i HlfViewer.obj
 0001:00001010       ?TextWidth@PluginDialogBuilder@@MEAAHAEBUFarDialogItem@@@Z 0000000180002010 f i HlfViewer.obj
 0001:00001020       ?DoShowDialog@PluginDialogBuilder@@MEAA_JXZ 0000000180002020 f i HlfViewer.obj
 0001:000010c0       ?SaveValue@PluginCheckBoxBinding@@UEAAXPEAUFarDialogItem@@H@Z 00000001800020c0 f i HlfViewer.obj
 0001:00001120       ?SaveValue@PluginRadioButtonBinding@@UEAAXPEAUFarDialogItem@@H@Z 0000000180002120 f i HlfViewer.obj
 0001:00001170       ??0PluginIntEditFieldBinding@@QEAA@AEBUPluginStartupInfo@@PEAPEAXHPEAHH@Z 0000000180002170 f i HlfViewer.obj
 0001:00001230       ?SaveValue@PluginIntEditFieldBinding@@UEAAXPEAUFarDialogItem@@H@Z 0000000180002230 f i HlfViewer.obj
 0001:00001280       ??0PluginUIntEditFieldBinding@@QEAA@AEBUPluginStartupInfo@@PEAPEAXHPEAIH@Z 0000000180002280 f i HlfViewer.obj
 0001:00001340       ?SaveValue@PluginUIntEditFieldBinding@@UEAAXPEAUFarDialogItem@@H@Z 0000000180002340 f i HlfViewer.obj
 0001:00001390       ?CreateCheckBoxBinding@PluginDialogBuilder@@MEAAPEAU?$DialogItemBinding@UFarDialogItem@@@@PEAHH@Z 0000000180002390 f i HlfViewer.obj
 0001:00001410       ?CreateRadioButtonBinding@PluginDialogBuilder@@MEAAPEAU?$DialogItemBinding@UFarDialogItem@@@@PEAH@Z 0000000180002410 f i HlfViewer.obj
 0001:00001480       ??_EPluginDialogBuilder@@UEAAPEAXI@Z 0000000180002480 f i HlfViewer.obj
 0001:00001480       ??_GPluginDialogBuilder@@UEAAPEAXI@Z 0000000180002480 f i HlfViewer.obj
 0001:000014d0       ?ShowHelp@@YA_NPEB_W0_N1@Z 00000001800024d0 f   HlfViewer.obj
 0001:00001590       SetStartupInfoW            0000000180002590 f   HlfViewer.obj
 0001:00001800       ?IsHlf@@YAHXZ              0000000180002800 f   HlfViewer.obj
 0001:00001a40       ?AddRadioButtons@?$DialogBuilderBase@UFarDialogItem@@@@QEAAXPEAHHQEBH_N@Z 0000000180002a40 f i HlfViewer.obj
 0001:00001c00       ?EndColumns@?$DialogBuilderBase@UFarDialogItem@@@@QEAAXXZ 0000000180002c00 f i HlfViewer.obj
 0001:00001d40       ?UpdateBorderSize@?$DialogBuilderBase@UFarDialogItem@@@@IEAAXXZ 0000000180002d40 f i HlfViewer.obj
 0001:00001e00       ?AddIntEditField@PluginDialogBuilder@@UEAAPEAUFarDialogItem@@PEAHH@Z 0000000180002e00 f i HlfViewer.obj
 0001:00001f10       ?AddUIntEditField@PluginDialogBuilder@@UEAAPEAUFarDialogItem@@PEAIH@Z 0000000180002f10 f i HlfViewer.obj
 0001:00002020       ?ShowCurrentHelpTopic@@YA_NXZ 0000000180003020 f   HlfViewer.obj
 0001:00002160       OpenW                      0000000180003160 f   HlfViewer.obj
 0001:00002620       ProcessEditorInputW        0000000180003620 f   HlfViewer.obj
 0001:000026e0       ConfigureW                 00000001800036e0 f   HlfViewer.obj
 0001:00003360       ??_U@YAPEAX_K@Z            0000000180004360 f   libCRT64:new_array.obj
 0001:00003370       wcschr                     0000000180004370 f   libCRT64:strchr.obj
 0001:00003390       memset                     0000000180004390 f   libCRT64:memset.obj
 0001:000033c0       ??_V@YAXPEAX@Z             00000001800043c0 f   libCRT64:delete_array.obj
 0001:000033d0       ??3@YAXPEAX@Z              00000001800043d0 f   libCRT64:delete.obj
 0001:000033e0       memcpy                     00000001800043e0 f   libCRT64:memcpy.obj
 0001:00003410       ??2@YAPEAX_K@Z             0000000180004410 f   libCRT64:new.obj
 0001:00003420       free                       0000000180004420 f   libCRT64:free.obj
 0001:00003450       malloc                     0000000180004450 f   libCRT64:malloc.obj
 0001:00003804       __IMPORT_DESCRIPTOR_KERNEL32 0000000180004804     kernel32:KERNEL32.dll
 0001:00003818       __IMPORT_DESCRIPTOR_RPCRT4 0000000180004818     rpcrt4:RPCRT4.dll
 0001:0000382c       __NULL_IMPORT_DESCRIPTOR   000000018000482c     kernel32:KERNEL32.dll

 entry point at        0000:00000000

 Static symbols

 0001:000007f0       ?frsuserfunc@@YAHPEBUPluginPanelItem@@PEB_WPEAX@Z 00000001800017f0 f   HlfViewer.obj
 0001:000015e0       ?ShowHelpFromTempFile@@YAXXZ 00000001800025e0 f   HlfViewer.obj
